:10000000D0C00000F3C00000F1C00000EFC000004D
:10001000EDC00000EBC00000E9C00000E7C0000038
:10002000E5C00000E3C000007CC30000E5C30000A1
:10003000DDC00000DBC00000D9C00000D7C0000058
:10004000D5C00000D3C00000D1C00000CFC0000068
:10005000CDC00000CBC00000C9C00000D1C200006C
:10006000C5C00000C3C00000C1C00000BFC0000088
:10007000BDC00000BBC00000B9C00000B7C0000098
:10008000B5C00000B3C00000B1C00000AFC00000A8
:10009000ADC00000ABC00000A9C00000A7C00000B8
:1000A000A5C00000A3C00000A1C000000001000026
:1000B000E2001200020000F4007300220100670158
:1000C0002100210100500109000300008801040102
:1000D0000309048C011201C13601C02601813601D9
:1000E00080361201000200000040C01685040001A5
:1000F0000001000109027300020100C0320904007E
:10010000000201030000072401000141000624024F
:100110000101000624020202000924030103010276
:100120000100092403020401010100090504024041
:1001300000000000052501010109058302400000BF
:10014000000005250101030904010002030000006D
:10015000092111010001222100070581034000014E
:100160000705020320000206C9FF0904A15C750807
:10017000150026FF009540097581029520097691AA
:100180000295040976B102C0040309041203590060
:100190006100790020004D00490044004900000042
:1001A000B30211241FBECFEFDAE0DEBFCDBF11E0F6
:1001B000A0E0B1E0E8E4FBE002C005900D92AE30B3
:1001C000B107D9F711E0AEE0B1E001C01D92AB3646
:1001D000B107E1F711E0C2EAD1E003C02297FE01C6
:1001E000ADD4C03AD107D1F749D0ACC409CF569AA3
:1001F000209A219A5E9A8CE091E09093610180931D
:100200006001089580910E016CE08AD4992311F069
:10021000299A0895299808951F93182F883FC1F4AB
:1002200080E090E02898289A019688309105D1F7CF
:10023000E9DF80910E018F5F80930E01883119F400
:1002400010920E015E9A80910E018C3009F45E9836
:1002500080910001181721F080910101181719F4FD
:1002600010920E015E9A80910201181709F45E98AF
:100270001F91089581E191E060E004C001D2B7DFF1
:10028000F9DFFECFFF920F931F93CF93DF93EC0123
:100290009FB7F89480916B01882311F49FBF2DC103
:1002A00084E08093E9002BE68091E80085FD07C09B
:1002B00082FF03C02093E800F7CF9FBF1DC12091AC
:1002C000F1003091F1000091F100F090F100809187
:1002D000E80085FD03C08BE68093E8009FBF922F66
:1002E0009F70892F8850883008F0ACC0132F1F7082
:1002F0001F5F662319F0611709F0FEC0832F807F0E
:10030000983059F4803809F0F7C01982CF5BDF4F7D
:10031000E881F981C154D0402BC09930E1F4803993
:1003200009F0EAC0FF2049F081E08983CD5BDF4F0F
:10033000E881F981C354D0401BC01982CF5BDF4FE5
:10034000E881F981C154D040309709F477C0812FFA
:10035000602F40E013C09A3099F4803A09F0CCC085
:1003600082E08983CB5BDF4FE881F981C554D040BF
:10037000309709F463C0812F602F4F2D09955EC01F
:100380009B3061F4803B09F0B7C083E08983C95B8F
:10039000DF4FE881F981C754D040EACF9C3061F447
:1003A000803C09F0A9C084E08983C75BDF4FE88106
:1003B000F981C954D0400DC09D3089F4803D09F0C9
:1003C0009BC085E08983C55BDF4FE881F981CB5411
:1003D000D040309799F1812F602F09952FC09E3022
:1003E000D9F4803E09F088C086E08983C35BDF4F83
:1003F000E881F981CD54D040309701F16F2D661F0F
:100400006627661F70E0802F90E08F779070682BD2
:10041000792B812F099512C09F3009F06DC0803F64
:1004200009F06AC088E08983C15BDF4FE881F98108
:10043000CF54D040309711F0832F099518830A8349
:10044000FB8258C0943021F5DE01A05CBF4F8C9137
:100450008C3330F4FE01E80FF11D34838F5F8C93F1
:10046000DE01A05CBF4F8C918C3330F4FE01E80FAD
:10047000F11D04838F5F8C93FE01E05CFF4F808150
:100480008C33D0F5C80FD11DFC828F5F808334C0C0
:10049000892F8550833080F5DE01A05CBF4F8C91A1
:1004A0008C3330F4FE01E80FF11D34838F5F8C93A1
:1004B000963060F0DE01A05CBF4F8C918C3330F43D
:1004C000FE01E80FF11D04838F5F8C93973061F478
:1004D000DE01A05CBF4F8C918C3330F4FE01E80F3D
:1004E000F11DF4828F5F8C93FE01E05CFF4F8081F1
:1004F0008A83108281E001C080E0DF91CF911F915B
:100500000F91FF90089580916B01882359F12FB7C7
:10051000F89481E08093E9009091E400975E31E0E7
:100520008091E80085FD0EC02FBF8091E4008917FF
:10053000C9F080916B018823A9F02FB7F89430930C
:10054000E900EECF6093F1008091E80085FD06C0E0
:100550008AE38093E80010926D0103C084E08093E9
:100560006D012FBF089587E091E090931001809373
:100570000F01E1E1F1E081E5DF011D928A95E9F7E4
:1005800008951DBA109268001CBC10BE1FBA1092CC
:100590007A0010926E0010926F001092710010920B
:1005A00072001092C900ECEBF0E0108214B817B89A
:1005B0001AB81DB810BA108215B818B81BB81EB8F2
:1005C00011BA0895F89480E29EE40197F1F781E072
:1005D0008093E00080E28093D8001092C90080E60A
:1005E0009AEE0197F1F7CDDF0C94003F0895F8944F
:1005F000C8DF80E69AEE0197F1F70C9400000895A9
:100600008F938FB78F9380916A018D5F8D37D0F470
:1006100080936A01809166018F5F80936601D8F0B4
:10062000809167018F4F80936701A8F080916801E6
:100630008F4F8093680178F0809169018F4F80938C
:10064000690109C08A5780936A01809166018E5FB3
:100650008093660128F7809162018C5F809362012C
:1006600058F0809163018F4F8093630128F080914F
:1006700064018F4F809364018F918FBF8F91189584
:10068000F894E1E6F0E020E82083108283E084BD66
:1006900085BDEEE6F0E080818160808391E09093FB
:1006A000800082E08093810090939000809391007D
:1006B0008093C00084E08093C1009093C200909327
:1006C000C3001092C40086E880937A0020937B00D8
:1006D00010927E0010927D0002D07894089580914F
:1006E000D80087FF02C085FF1BC081E08093D70040
:1006F00080EA8093D80082E189BD09B400FEFDCF75
:1007000080E98093D8001092E00010926B01109263
:100710006C0110926D011092E1008CE08093E20078
:1007200008951F920F920FB60F9211248F939F93EB
:100730008091E1001092E100982F83FF0FC010928A
:10074000E90081E08093EB001092EC0082E380935B
:10075000ED0088E08093F00010926B0192FF24C0BE
:1007600080916B01882301F180916D01882391F0C4
:10077000815080936D01882369F481E08093E900C2
:1007800002C01092F1008091E80085FDFACF8AE363
:100790008093E80083E08093E9008091F200882351
:1007A00019F08AE38093E80090FF0CC080E1809309
:1007B000E20010926B0181E080936C0180EA8093EB
:1007C000D80019BC80916C01882379F094FF0DC08A
:1007D00082E189BD09B400FEFDCF80E98093D80095
:1007E0008DE08093E20010926C019F918F910F90A9
:1007F0000FBE0F901F9018951F920F920FB60F9279
:1008000011242F933F934F935F936F937F938F9315
:100810009F93AF93BF93EF93FF931092E900809162
:10082000E80083FF32C13091F1009091F1004091D6
:10083000F1005091F1006091F1007091F100A091F0
:10084000F100B091F10082EF8093E800963009F05A
:1008500044C0ECEAF0E020E085919591841795077B
:1008600011F0359617C0859195918617970711F06D
:10087000339610C0259135914491CD01AF3FB1051C
:1008800019F010F08FEF90E0841708F4482FF90169
:100890005EEF04C02F5F2630F9F6F7C08091E800C4
:1008A000282F30E0C90185709070892BB9F322FDA3
:1008B000EFC0242F413408F020E4922F04C085912A
:1008C0008093F10091509923D1F7421B5093E80097
:1008D000442321F7203411F3DBC0953061F48EEF0F
:1008E0008093E8008091E80080FFFCCF842F80682F
:1008F0008093E300CDC09930F9F4332309F06FC041
:1009000040936B0110926D018EEF8093E800E6ED4D
:10091000F0E091E09093E90085918093EB008823CB
:1009200031F085918093EC0085918093ED009F5F7D
:10093000953081F78EE14EC0983061F4303809F07F
:100940004EC08091E80080FFFCCF80916B018093C6
:10095000F1001BC09923E9F48091E80080FFFCCFEF
:10096000323811F080E00DC06093E9008091EB0017
:1009700090E025E0969587952A95E1F78170109291
:10098000E9008093F1001092F1008EEF8093E8006F
:100990007FC0913011F0933011F5323001F54115DF
:1009A0005105E9F4262F2F77822F81508430B8F437
:1009B0008EEF8093E8002093E900933009F465C03E
:1009C00089E18093EB0081E090E002C0880F991FDD
:1009D0002A95E2F78093EA001092EA0059C061304C
:1009E000710509F052C0913019F5313A09F04DC046
:1009F0004A2F5EEF8091E800282F30E0C901857012
:100A00009070892BB9F322FD43C0942F413408F034
:100A100090E4892F03C01092F10081508823D9F708
:100A2000491B5093E800442329F7903419F330C050
:100A3000993059F5313249F54050534031F514970A
:100A400021F58091E80082FFFCCF9091F100209188
:100A5000F1003091F1004091F1008BEF8093E800BC
:100A60008EEF8093E800993A39F4253471F4323CE2
:100A700061F44B3651F4A6DD9B3839F4253C29F45A
:100A80003D3119F4403709F4B2DD81E28093EB0087
:100A9000FF91EF91BF91AF919F918F917F916F9156
:100AA0005F914F913F912F910F900FBE0F901F902C
:100AB00018950F931F93CF93DF938C01EB0109C01F
:100AC0002196D801ED91FC910190F081E02DC801B3
:100AD000099568816623A1F7DF91CF911F910F914E
:100AE0000895EF92FF920F931F93CF93DF938C01A2
:100AF0007B01EA010CC0D7016D917D01D801ED9118
:100B0000FC910190F081E02DC80109952197209773
:100B100091F7DF91CF911F910F91FF90EF90089582
:100B2000991B79E004C0991F961708F0961B881F3F
:100B30007A95C9F780950895EE0FFF1F0590F491FF
:080B4000E02D0994F894FFCFA9
:0E0B4800FAFBFC000000008302590571050055
:00000001FF
